:020000000126D7
:03000300024003B5
:03000B0002400BA5
:0300130002401395
:03001B0002401B85
:1000230002402375817053D0E775A80075A2F09044
:10003300BF8074007E13F0A3DEFC90BF907400F0C9
:10004300A37440F090BF927470F074FA90BF93F071
:1000530041248E7E8F7FE5A61340FB7E44DEFE7F28
:1000630008C0E0E5A613D0E0137E2CDEFEDFF2C36A
:10007300AF7FAE7E228E7E8F7F75A67F7E2EDEFEC5
:100083007F0813400575A67F800575A6FF80007E57
:100093002BDEFEDFED75A6FF7E2FDEFEAF7FAE7E8D
:1000A30022046A0000000000031200C13830353119
:1000B300206D6F6E69746F722056312E3200C0E06E
:1000C3007401C0A8C2AFC083C08290BF80F0A37484
:1000D30000F0A3E5D0F0A3D0E0F0A3D0E0F0A3D0EC
:1000E300E0F0A3D0E0F0A3E5F0F0A3716390BF804C
:1000F300E0F8D0E0F9D0E0B8010524FD4001199003
:10010300BF90F0A3E9F0A3E581F0412490BF9311E0
:100113005540F9B4F70040F4F0A3115540EEB46B29
:100123000050E9F0A36009FE115540E0F0A3DEF8AA
:10013300115540D8FD71502D70D290BF93E0FEA3AE
:10014300E0CEA3B4FF02217DB4FE02219BB4FD02E5
:1001530021C9B4FC024124B4FB02414BB4FA02416D
:100163008EB4F90241C4B4F8026103B4F702611416
:1001730074F090BF93F07401612C90BF94741DF0E0
:10018300A3FE7F00A882A9839000A4EF930F888227
:100193008983F0A3DEEE6138A3E0F8A3E0F9A3E0DE
:1001A300FE90BF94F0A3601CAA82AB8388828983EC
:1001B300B90003E68001E0A3A882A9838A828B8326
:1001C300F0A3DEE46138A3E0F8A3E0F9A3EE24FD95
:1001D3006047FEFFE0AA82AB8388828983B900036C
:1001E300F68001F0A3A882A9838A828B83A3DEE42D
:1001F30090BF96E0F8A3E0F9A3E0FEAA82AB838860
:10020300828983B90003E68001E06E7010A3A8829F
:10021300A9838A828B83A3DFE07400800274016167
:100223002C90BF807413FEA882A98390BF94F0A37F
:10023300AA82AB8388828983E0A3A882A9838A8266
:100243008B83F0A3DEEA6138EE603EA3A3E054188B
:10025300F5F065D05418601190BF9D717C53D0E7C1
:10026300E5F042D090BF9D7163788079BF90BF94D1
:10027300E0FEA3E0A3AA82AB8388828983F0A3A8CC
:1002830082A9838A828B83DEEA412490BF92E0F5C0
:100293008190BF88717CE0C0E0A3E0C0E090BF859F
:1002A300E0C0E0A3E0C0E0A3E0F5F0A390BF82E0EC
:1002B300F5D0A3E0C0E0A3E0F583D082D0E0D0A8DE
:1002C30022EE6032AA82AB83AC82AD838A828B83B7
:1002D300A3E0F8A3E0F9A3E0FFA3AA82AB8388829B
:1002E3008983E0F8EFF0E08C828D836F7008E8F08B
:1002F300A31E1E1EDED2E582246B90BF94F06138EC
:10030300E0F874E5F0A3E8F0A37422F012BF95615E
:100313002CE0F8A3A3E0F974F5F0A3E8F0A37422AA
:10032300F0E912BF977400612CF890BF947401F048
:10033300A3E8F08000715064FF04F090BF94E024C0
:1003430003FE90BF93E01178A3DEFA210F90BF94D0
:10035300E02402FE90BF937F00E02FFFA3DEFA228A
:10036300E8F0A3E9F0A3EAF0A3EBF0A3ECF0A3ED2C
:10037300F0A3EEF0A3EFF0A322E0F8A3E0F9A3E0EB
:10038300FAA3E0FBA3E0FCA3E0FDA3E0FEA3E0FFF0
:02039300A322A3
:00002601D9
